:1000000012C0189518951895189518951895189563
:1000100018956BC0189518951895189518951895FA
:100020001895189518958FE58DBFC0E4E8E34E2E1E
:1000300084E08EBFD4E0F4E05F2EEEEFF3E0A0E6C4
:10004000B0E0A89584B7082E877F84BF88E1992700
:1000500081BD91BD88278D933197E9F7662480E0B3
:1000600087BB8FEF88BB8FEF84BB80EF85BB8FEFA3
:1000700081BB8FEF82BB84E083BF89B7816089BF7A
:100080007894E1E0F0E0A2E6B0E091E0B8D200912F
:100090006200033680E010F009F081E08F93009158
:1000A0006200013081E008F080E09F91892B882375
:1000B00009F403C088E28093620080E080936300CB
:1000C0000027A1E6B0E08C9187FB0EF401E041E04F
:1000D000041709F007C0809161008F778093610059
:1000E000A5D079D1EDCFF894FFCF0F921F922F9228
:1000F0003F924F925F927F92AF92BF920F931F9366
:100100002F933F934F935F936F937F938F939F931F
:10011000AF93BF93CF93DF93EF93FF938FB78F93FB
:1001200086E0809352008091610080688093610036
:10013000A0E6B0E08C918F5F8C93009160000A3F45
:1001400009F058C080E080936000A1E6B0E08C9197
:1001500084FB882780F9809580FBA1E6B0E08C9134
:1001600084F98C930027A1E6B0E08C9182FB0EF419
:1001700001E041E0041709F038C0A1E6B0E08C913D
:1001800084FBA1E6B0E08C9186F98C9380916300AA
:10019000815080936300009163000F3F09F008C015
:1001A0008BE38093630080916200815080936200B2
:1001B00000916200003081E009F080E08F930091AF
:1001C0006300003081E009F080E09F91892388235B
:1001D00009F40AC0809161008B7F80936100809157
:1001E000610082608093610005C0809161008F7B17
:1001F000809361008F918FBFFF91EF91DF91CF913D
:10020000BF91AF919F918F917F916F915F914F912E
:100210003F912F911F910F91BF90AF907F905F9072
:100220004F903F902F901F900F901895A8E6B0E048
:100230008C918F5F8C9300916800043009F003C0AB
:1002400080E08093680000916800003009F012C0DF
:10025000A898009162004AE0D9D1A7E6B0E00C93DB
:1002600000916700003009F003C08AE080936700C6
:10027000AB9A26C0013009F00AC0AB980091620029
:100280004AE0C4D1A7E6B0E08C93AA9A19C0023024
:1002900009F00AC0AA98009163004AE0B7D1A7E626
:1002A000B0E00C93A99A0CC0033009F009C0A998DA
:1002B000009163004AE0AAD1A7E6B0E08C93A89A27
:1002C0000027A1E6B0E08C9181FB0EF401E040E054
:1002D000041709F00AC0E6E8F5E0A7E6B0E08C9163
:1002E0009927A7E6B0E06ED112C00027A1E6B0E0E2
:1002F0008C9184FB0EF401E041E0041709F004C086
:100300008FEB8093670003C08FEF80936700002717
:10031000A1E6B0E08C9185FB0EF401E041E004170A
:1003200009F003C08FEF80936700A7E6B0E08C91DF
:1003300084FBA5E3B0E08C9184F98C93A7E6B0E050
:100340008C9183FBA5E3B0E08C9185F98C93A7E6B3
:10035000B0E08C9182FBA5E6B0E08C9180F98C93A3
:10036000A7E6B0E08C9186FBA5E6B0E08C9181F920
:100370008C93A7E6B0E08C9185FBA5E6B0E08C916C
:1003800082F98C93A7E6B0E08C9180FBA5E6B0E003
:100390008C9183F98C93A7E6B0E08C9181FBA5E664
:1003A000B0E08C9184F98C93A1E6B0E08C9186FB4F
:1003B000A5E6B0E08C9185F98C93A1E6B0E08C9134
:1003C00083FBA5E6B0E08C9186F98C93A5E6B0E0BE
:1003D0008C9182BB089506B347E00423AAE6B0E0FF
:1003E0000C9300916A00073081E009F480E08F935C
:1003F00040916A0000916900041781E009F080E0F3
:100400009F918923882309F4B6C0ABE6B0E08C91B4
:100410008F5F8C9300916B00043609F0ABC080E0D5
:1004200080936B000027A1E6B0E08C9181FB0EF475
:1004300001E040E0041709F079C00091690006303E
:1004400009F019C00027A1E6B0E08C9182FB0EF400
:1004500001E040E0041709F00DC00091620003368E
:1004600008F005C0A2E6B0E08C918F5F8C9380E02D
:10047000809363005AC0053009F01BC00027A1E635
:10048000B0E08C9182FB0EF401E040E0041709F02B
:100490000FC000916200013010F009F001C005C0EA
:1004A0008091620081508093620080E080936300BD
:1004B0003CC0033009F01FC00027A1E6B0E08C91DA
:1004C00085FB0EF401E040E0041709F00EC0A1E640
:1004D000B0E08C9182FB882780F9809580FBA1E6B3
:1004E000B0E08C9182F98C9305C0809161008F7D82
:1004F000809361001AC0043009F017C00027A1E6FC
:10050000B0E08C9182FB0EF401E040E0041709F0AA
:100510000CC0E1E0F0E0A2E6B0E091E07BE75ED065
:100520008091610080628093610024C080916100AD
:100530008D7F80936100E1E0F0E0A2E6B0E091E021
:100540005ED000916200033680E010F009F081E097
:100550008F9300916200013081E008F080E09F916C
:10056000892B882309F403C088E28093620080E02D
:100570008093630007C080916A00809369008CE3D8
:1005800080936B000895C0F9A4B0999282F880908E
:10059000FFBF3197F1F70895689462F80895E894E1
:1005A00062F80895C89531960020089591E005C03D
:1005B00092E003C094E001C098E0F4DF0D929A95B8
:1005C000E1F70895E80FF91FF1CFE199FECFEEBBF7
:1005D000FFBB3196089591E001C092E07B3751F462
:1005E0007FB7F894F2DF8D918DBBE29AE19A9A95EC
:1005F000C9F77FBF7727089591E001C092E0E5DF5A
:10060000E09A8DB38D939A95D1F70895FF93881B47
:10061000F9E0001FFA9511F4FF910895881F841BDB
:0C06200018F4840F8894F5CF0894F3CFF1
:00000001FF
